:10099100232132303045465500232432303045463C
:0209A1005500FF
:10096600AF8475840F758A83E4F58475C04475CFAA
:05097600E4C2C38F8400
:01097B002259
:060912008F27AD27AF2680
:020918008D1E32
:10091A001208F0EFC454F0F51FAF1E1208F0EF25CD
:04092A001FF51FFF97
:01092E0022A6
:1008C9008F828E83D3E5829DE5839C501943B701BE
:1008D900758F03E4F0F58F53B7FE2582F582740412
:0608E9003583F58380DE7B
:0108EF0022E6
:0206D800A90770
:1006DA0020C3FD20C5FAC2C4D2C5E4FFFC30C3FD65
:1006EA0030C3FDE5C154F8FA64086003BA1011E595
:1006FA001DBF01044401800254FEF5C27C01807CC6
:10070A00BA180B851CC27C02C2C4C2C5806EBA204C
:10071A00028038EA64287030B9010CBC02028015E4
:10072A00EC6404701F8019BC02088BC27C03C2C52A
:10073A008012BC03088DC27C04C2C58007BC0404B5
:10074A00D2C57F01C2C48034BA300AD2C4D2C57CB1
:10075A0009E4FF8027BA3802801EBA4006C2C2C224
:10076A00C58019BA48028010BA50028003BA5808E4
:10077A00D2C47C08AEC28004D2C4D2C5C2C3EC645F
:08078A000860030206EAAF0655
:010792002244
:1009B400AE05AD078E1C8B1DE4FB7F011206D82209
:1009A300AE03AB05AD078E1C751DA07F021206D8E2
:0109B3002221
:0603B2008B3D8A3E893FED
:1003B8007547FF754809754991754401754500757C
:1003C8004600E4F543F542F541F540E47F50FEFD73
:1003D800FCAB43AA42A941A840C312066C5031AFF6
:1003E800437BA0E4FD1209B47844E475F0011206D9
:1003F800C8EF12064DAF43AE42AD41AC40E47B01BD
:10040800FAF9F812065F8F438E428D418C4080BB0B
:10041800AB47AA48A949120607FF900000E06F7091
:1004280062900001120620FF900001E06F70549066
:100438000002120620FF900002E06F704690000351
:10044800120620FF900003E06F7038900004120637
:1004580020FF900004E06F702A900005120620FF2C
:10046800900005E0B5071C900006120620FF9000DA
:1004780006E0B5070E900007120620FF900007E07F
:100488006F60037F0022AB3DAA3EA93F120607FF1B
:10049800900011E06F702A900001120620FF900072
:1004A80012E0B5071C900002120620FF900013E02E
:1004B800B5070E900003120620FF900014E06F604D
:1004C800037F0022900009E0F55BA3E0F55DA3E05F
:1004D800F55E900019E0F557A3E0F559A3E0F55A49
:0204E8007F0192
:0104EA0022EF
:0D092F008F0DAF18AE1712097C8E178F18B0
:02093C00AC0607
:0D093E00AB07AF04AD07AF03AB581209B40F
:01094B002289
:0E09E200E55CC3955B500605580558055C2280
:10097C000FBF00010ED3EF955EEE955D4006120998
:05098C00E2E4FEFF2281
:040277008E088F0955
:10027B00E4F50DF50EF513F514F515F516F517F563
:10028B0018855917855A18855758F50EF50D755C55
:10029B0001E4F512E50D643A6016AF18AE171209BA
:1002AB003C8F0DAF18AE1712097C8E178F1880E498
:1002BB000514E51470020513AF18AE1712093C12A2
:1002CB00092F8F0EAD0EAF0D1209188F108510125E
:1002DB0012093112092F8F0EAD0EAF0D12091875C1
:1002EB0015008F16EF2512F512E516751600F5158C
:1002FB0012093112092F8F0EAD0EAF0D120918EF27
:10030B00421685150A85160BE5162512F5121209EC
:10031B003112092F8F0EAD0EAF0D1209188F0FE58D
:10032B000F2512F512E50F705CF50CE50CC395105B
:10033B00505312093112092F8F0EAD0EAF0D12094A
:10034B00188F11E5112512F512C3E50B9509E50A76
:10035B009508402DAE0AAF0BBEFB06BFFE0343B1A3
:10036B003043B701758F01850B82850A83E511F048
:10037B00E4F58F53B7FE75B111050BE50B70020554
:10038B000A050C80A612093112092F8F0EAD0EAF84
:10039B000D1209188F11E5112512700AE50F640172
:0603AB00600302029C2227
:0103B1002229
:0604EB008B4A8A4B894C8C
:1004F1007554FF75550975569A75510175520075F8
:100501005350E4F550F54FF54EF54DE47F2BFEFDCC
:10051100FCAB50AA4FA94EA84DC312066C5030AF88
:1005210050E4FBFD1209A37851E475F0011206C8ED
:10053100EF12064DAF50AE4FAD4EAC4DE47B01FA1C
:10054100F9F812065F8F508E4F8D4E8C4D80BCABEB
:1005510054AA55A956120607FF900050E06F706229
:10056100900001120620FF900051E06F705490003E
:1005710002120620FF900052E06F704690000312B5
:100581000620FF900053E06F70389000041206209F
:10059100FF900054E06F702A900005120620FF9032
:1005A1000055E0B5071C900006120620FF9000568A
:1005B100E0B5070E900007120620FF900057E06F8C
:1005C10060037F0022AB4AAA4BA94C120607FF9099
:1005D100005FE06F702A900001120620FF9000601A
:1005E100E0B5071C900002120620FF900061E0B503
:1005F100070E900003120620FF900062E06F600377
:050601007F00227F01D3
:0106060022D1
:10085800E48F34F533F532F531AE33AD32AC31785F
:10086800081206958F348E338D328C317835120606
:01087800A8D7
:080879008F628E618D608C5FBF
:10088100AA077808120682A907AF62AE61AD60AC13
:0F0891005F7810120682AB07AF02AD011209A308
:0108A0002235
:0400A6008E218F22F6
:1000AA00E4F526F527F534F533F532F531F538F56B
:1000BA0037F536F535F53CF53BF53AF53975382B14
:1000CA00F537F536F535F527F526F52CE4F52BE564
:1000DA0026643A60071208748F2680F3E53C2401EF
:1000EA00FFE4353BFEE4353AFDE435398F3C8E3B7F
:1000FA008D3AF5391208748F261208741209128F74
:10010A002985292B1208748F26120874120912E401
:10011A008F30F52FF52EF52DEF252BF52BAE2FADC4
:10012A002EAC2D78081206958F308E2F8D2E8C2DA1
:10013A001208748F26120874120912E5304FFFE56F
:10014A002FFEE52EFDE52D8F308E2F8D2EF52D8E6F
:10015A00238F24EF252BF52B1208748F261208748F
:10016A001209128F28E528252BF52BE5286404703F
:10017A00381208748F261208741209121208588F3E
:10018A0026120874120912E5344FFFE533FEE532F0
:10019A00FDE5318F348E338D32F531FC781012063D
:1001AA00958F348E338D328C31E528640270381283
:1001BA0008748F261208741209121208588F261210
:1001CA000874120912E5344FFFE533FEE532FDE506
:1001DA00318F348E338D32F531FC78041206958FC7
:1001EA00348E338D328C31E5342524F524E53335CC
:1001FA0023F523E5287058F525E525C39529504FA1
:10020A001208748F261208741209128F2AE52A25F9
:10021A002BF52BC3E5249522E5239521402DAE230A
:10022A00AF24BEFB06BFFE0343B13043B701758F4F
:10023A0001852482852383E52AF0E4F58F53B7FEEE
:10024A0075B1110524E52470020523052580AA123B
:10025A0008748F261208741209128F2AE52A252B90
:0C026A00700AE528640160030200D6223F
:010276002265
:05000600323530450019
:1008A10075840F75A4CF75A71C75B0E7E4F5E275E3
:1008B100A6FF75E10375E3C0F5A57590FF75ADE37E
:0808C10075AD63F5A5F5842275
:0F09C400E4F584759A4075F809759D01F5842254
:0609F0001209660209C4B1
:0F09D3001208A1E5B05402FFEF7002D322C32235
:10079300C200C201C20275FFDE75FFAD1209D3921A
:1007A3000030005E1209F07BFF7A0079061203B273
:1007B300EF24FF92013001147D007CA07F007E4076
:1007C3001208C97F007E4012027780237BFF7A00E4
:1007D30079061204EBEF24FF92023002127D007CB3
:1007E300A07F007E401208C97F007E401200A6E46D
:1007F300FFFE0FBF00010EBE27F8BF10F5E4F5841E
:05080300F5C002000E2B
:04000E00024000228A
:01FBFE00FE08
:0300000002094CA6
:03000300025003A5
:03000B000250069A
:030013000250098F
:03001B0002500C84
:0300230002500F79
:03002B000250126E
:0300330002501563
:03003B0002501858
:0300430002501B4D
:03004B0002501E42
:0300530002502137
:03005B000250242C
:0300630002502721
:03006B0002502A16
:0300730002502D0B
:03007B0002503000
:03008300025033F5
:03008B00025036EA
:03009300025039DF
:03009B0002503CD4
:0300A30002503FC9
:10094C00787FE4F6D8FD9000007F007E20E4F0A3D1
:0A095C00DFFCDEFA758162020793EA
:10080800E590540C23C0E0740AC0E0C082C08302A3
:100818000A00E590540C23C0E0740AC0E0C082C00E
:1008280083020A08E590540C23C0E0740AC0E0C0B3
:1008380082C083020A10E590540C23C0E0740AC0F9
:08084800E0C082C083020A181F
:040A00005390F322FA
:070A080043900C5390F7220C
:070A100043900C5390FB2200
:040A180043900C22D9
:07085000EFC403900A0073DE
:10060700BB010689828A83E0225002E722BBFE02F1
:09061700E32289828A83E4932224
:10062000BB010CE58229F582E5833AF583E022508F
:1006300006E92582F8E622BBFE06E92582F8E222D9
:0D064000E58229F582E5833AF583E49322F3
:10064D00BB010689828A83F0225002F722BBFE018C
:02065D00F32286
:0D065F00EF2BFFEE3AFEED39FDEC38FC22EA
:10066C00EB9FF5F0EA9E42F0E99D42F0EC6480C805
:06067C0064809845F022A5
:10068200E8600FECC313FCED13FDEE13FEEF13FF56
:03069200D8F1227A
:10069500E8600FEFC333FFEE33FEED33FDEC33FCC3
:0306A500D8F12267
:1006A8007401FF3395E0FEFDFC080808E6CF2FF63D
:1006B80018E6CE3EF618E6CD3DF618E6CC3CF62216
:1006C800FAE6FB0808E6F925F0F618E6CA3AF62233
:1008F000EF7E0024D0B40A00401624F9B40A004068
:100900000CB41000400A24E0B41000400374FFFE51
:02091000FF22C4
:00000001FF
